:020000040000FA
:10000000BE280400000000003E2400003E24000042
:100010003E2400003E2400003E2400003E24000058
:100020003E2400003E2400003E2400003E24000048
:100030003E2400005A2400003E2400003E2400001C
:100040003E2400003E2400003E2400003026000034
:100050003E2400003E2400003E2400003E24000018
:100060003E2400003E2400003E2400003E24000008
:100070003E2400003E2400003E2400003E240000F8
:100080003E2400003E2400003E2400003E240000E8
:100090003E2400003E2400003E2400003E240000D8
:1000A0003E2400003E2400003E2400003E240000C8
:1000B0003E2400003E2400003E2400003E240000B8
:1000C0003E2400003E2400003E2400003E240000A8
:1000D0003E2400003E2400003E2400003E24000098
:1000E0003E2400003E2400003E2400003E24000088
:1000F0003E2400003E2400003E2400003E24000078
:100100003E2400003E2400003E2400003E24000067
:100110003E2400003E2400003E2400003E24000057
:100120003E2400003E2400003E2400003E24000047
:100130003E2400003E2400003E2400003E24000037
:100140003E2400003E2400003E2400003E24000027
:100150003E2400003E2400003E2400003E24000017
:100160003E2400003E2400003E2400003E24000007
:100170003E2400003E2400003E2400003E240000F7
:100180003E2400003E2400003E2400003E240000E7
:100190003E2400003E2400003E2400003E240000D7
:1001A0003E2400003E2400003E2400003E240000C7
:1001B0003E2400003E2400003E2400003E240000B7
:1001C0003E2400003E2400003E2400003E240000A7
:1001D0003E2400003E2400003E2400003E24000097
:1001E0003E2400003E2400003E2400003E24000087
:1001F0003E2400003E2400003E2400003E24000077
:10020000B6280000000000008344550050000000A4
:1002100000277800000006000A0000008444520015
:100220004F5000003E007800000006000A00000069
:1002300084535700414200000080FD00000006008A
:100240000A000000834E4900500000000E87E800BD
:10025000000006000A000000C4545500434B000093
:100260001E27780010079800000006000C00000010
:10027000C4535700415000009E1F7800000F7800C3
:100280004F007800000006000E000000C44F56002A
:1002900045520000002778001E0090000000060074
:1002A0000C000000C3524F0054000000801F780073
:1002B0001E0090003E0F78004F27780000000600D7
:1002C00010000000C4504900434B00000000E9004A
:1002D000000040006E007800000006000E000000E4
:1002E000C4504F004B4500000000E90000004000F2
:1002F0000E0040003E0878003E0078000000060036
:1003000012000000C4524F004C4C00000000E900F5
:100310000C003400811F7800821F78008E0040009E
:1003200081004000911F7800010178000000E90081
:1003300000800900C21078004F0F78004F0178004C
:10034000CF0078003E007800000006002600000084
:10035000C43F4400555000000000B00001003200CE
:1003600000277800000006000E000000823E5200C8
:10037000801F78003E007800000006000A000000A0
:1003800082523E00002778004F00780000000600EF
:100390000A00000082524000002778007FB89700D2
:1003A000000006000A0000008140000010007800F4
:1003B0000000060008000000C24340001040780022
:1003C0000000FB00000006000A000000C121000040
:1003D0003E0878003E007800000006000A00000099
:1003E000C24321001E4878003E0078003E0078009D
:1003F000000006000C000000812B00003E004000C1
:100400000000060008000000C22B2B00811F7800AE
:10041000BE0078003E0040001E8F4800CF007800EC
:100420000000060010000000864E450047415400C1
:10043000450000000000EA00000006000C0000007B
:10044000812D00003E0010000000060008000000A2
:10045000C22D2D00811F7800BE0078003E001000E4
:100460001E8F1800CF00780000000600100000006A
:1004700082322A004100DD00000006000800000072
:1004800082342A004200DD0000000600080000005F
:1004900082322F004180DE000000060008000000CC
:1004A00082342F004280DE000000060008000000B9
:1004B00082303C004F80DE00000006000800000093
:1004C000C2303D000000B000010032000080EF00AB
:1004D0000080EA00000006000E000000C2303E006E
:1004E0000000B000020032000080EA004F80DE0011
:1004F000000006000E000000C2553C003E00100047
:100500000000EF00F2FF3900000006000C000000C0
:10051000C13C00003E0010000000EF00ECFF350081
:10052000000006000C000000C13D00003E00680015
:100530000000EF00E6FF3200000006000C000000A3
:10054000C13E00003E0010000000EF00E0FF3C0054
:10055000000006000C000000C34E4F0054000000D5
:100560000000B000DAFF32000000EF0000000600DB
:100570000E000000C2552A00811F78003E00B8001E
:10058000CF007800000006000C000000C12A000027
:10059000811F78003E80B900CF007800000006007F
:1005A0000C000000C5552F004D4F4400821F7800FD
:1005B000811F7800000178001E00780011000900FA
:1005C0000280D800010F7800CF0078004F0178003A
:1005D000000006001A000000C6552A002F4D4F00EB
:1005E00044000000821F7800811F7800000178001D
:1005F0003E0078001E00B800110009004288D800B3
:10060000010F7800CF0078004F017800000006004D
:100610001E000000C52A2F004D4F4400821F7800A5
:10062000811F7800000178003E0078001E80B9002C
:10063000110009004208D800010F7800CF007800AF
:100640004F017800000006001C000000C42F4D0080
:100650004F440000821F7800811F7800000178005D
:100660001E007800110009000200D800010F780078
:10067000CF0078004F017800000006001A0000004B
:10068000C12F0000811F780080007800F1FF070073
:1006900001F0A300010039008100EA00801F78000A
:1006A0003E00780000F0A300010039000000EA00DD
:1006B0004100DD00810050004F007800CF0078003D
:1006C0000500390000F0A300020031000000E8003E
:1006D000000006000000E9000000060030000000F5
:1006E000C34D4F0044000000DAFF07003E007800D1
:1006F000000006000C000000C22A2F00811F7800B5
:1007000080007800C5FF0700E1FF37000000060009
:100710000E000000C453510052540000831F7800A3
:10072000821F7800811F78000027EB00010820005D
:100730001E8140000211B8000200E10001003900F2
:100740001E8F40008100D100F9FF39001E01E80032
:100750001E11B8000010E100010031001E0FE8007A
:10076000CF0078004F017800CF0178003E0078007C
:100770000000060032000000C34D41005800000098
:100780001E00E10002003C003E0078000000060070
:10079000620747000000060012000000C34D490038
:1007A0004E0000001E00E100F9FF35003E00780019
:1007B000000006000E000000C3414200530000008C
:1007C0000000B00001003B000000EA00000006004D
:1007D0000E00000083414E00440000003E00600017
:1007E000000006000A000000824F52003E00700028
:1007F000000006000800000083584F00520000006F
:100800003E006800000006000A000000C3415300DB
:10081000480000000000B0000800320004003B0067
:100820000080EA00008009001E8FD100030037001D
:100830000000E900008009001E0FD0003E00780093
:10084000000006001E000000C34C530048000000DA
:100850000000B000F9FF3200F5FF3B000080EA0025
:10086000008009001E0FD100F4FF370000000600D1
:1008700016000000C3524F004C0000000000B00002
:10088000EEFF320004003B000080EA000080090017
:100890001E0FD300E9FF37000000E90000800900C7
:1008A0001E0FD200E5FF3700000006001E0000000A
:1008B00083434F004D0000000080EA000000060066
:1008C0000A000000C32B430021000000811F7800B4
:1008D000BE00780010C840003E007800CF007800CD
:1008E0000000060012000000C32D4300210000009C
:1008F000811F7800BE00780010C810003E0078000C
:10090000CF0078000000060012000000C22B21007A
:10091000811F7800BE007800108840003E007800FB
:10092000CF0078000000060010000000C22D21005A
:10093000811F7800BE007800108810003E0078000B
:10094000CF0078000000060010000000C4464900F7
:100950004C4C0000821F7800811F78003E01780017
:10096000BE0078000201E90002800900805878008A
:100970003E007800CF0078004F01780000000600AC
:100980001C000000C5434D004F564500821F7800F3
:10099000811F78003E0178009E001100BE007800A3
:1009A000050039000000E90009003300008009005B
:1009B00031597800060037000201400081004000F4
:1009C0000000E90002003300008009004161780066
:1009D0003E007800CF0078004F017800000006004C
:1009E00030000000C44D4F0056450000821F7800C3
:1009F000811F78003E0178009E001100BE00780043
:100A0000050039000000E9000B00330000800900F8
:100A1000311978000800370002014000020140004F
:100A200081004000810040000000E9000200330026
:100A300000800900412178003E007800CF00780056
:100A40004F01780000000600340000008449440093
:100A50004C4500000140FE00000006000A000000B6
:100A600085534C00454550000040FE000000060044
:100A70000A000000C8535F0054414D00504F4E0023
:100A80000027780000802000000006000E00000013
:100A9000C6535F00574F5200440000000027780003
:100AA00000862000000006000E000000C8535F0012
:100AB000464F52004D41540000277800008A200024
:100AC000000006000E000000C549540052583100D5
:100AD0000027780000902000000006000C000000B5
:100AE000C55445004C454300002778004090200045
:100AF000000006000C000000C6434E00544954009C
:100B000050000000002778006090200000000600E0
:100B10000E000000C3504100440000000027780090
:100B200020912000000006000C000000C33E490098
:100B30004E000000002778004091200000000600D1
:100B40000C000000C94D45004D5F44004550540065
:100B50004800000000277800609120000000060097
:100B600010000000CB4D45004D5F5000524748003B
:100B700045524500002778008091200000000600C3
:100B800010000000CA414400525F4300524541003A
:100B90005445000000277800C091200000000600A6
:100BA00010000000C5535400415254000027780043
:100BB00000922000000006000C000000C554450013
:100BC0004D5053000027780040922000000006009E
:100BD0000C000000C5544100434845000027780040
:100BE00060922000000006000C000000C84D450087
:100BF0004D5F480045524500002778008092200054
:100C0000000006000E000000CA5354004F505F0061
:100C1000464F52005448000000277800A092200060
:100C20000000060010000000C4454F004C4E0000BC
:100C300000277800E0922000000006000C00000071
:100C4000C3454F00460000000027780000932000B5
:100C5000000006000C000000C442410053450000A3
:100C60000027780020932000000006000C00000000
:100C7000C55354004154450000277800409320009C
:100C8000000006000C000000C5455200524F520003
:100C90000027780060932000000006000C00000090
:100CA000C9545F005355530050454E0044000000A6
:100CB00000277800C093200000000600100000000C
:100CC000C8505200494F520049544500002778004F
:100CD000E0932000000006000E000000CA494E000C
:100CE000505554005F4649004C45000000277800ED
:100CF000009420000000060010000000C7505200C1
:100D0000475F50004E54000000277800409F2000AD
:100D1000000006000E000000C54445005054480085
:100D200000277800E0DF20000E0050004180DE0048
:100D30000000060010000000C65244004550540058
:100D4000480000000027780040D0200000805700B5
:100D50004180DE000000060012000000C750520073
:100D6000474845005245000082FF070000277800F1
:100D7000801F78003E0078002000B000100078004E
:100D8000002778004F00780010007800000006006F
:100D90001C000000C83E5000524748004552450024
:100DA00074FF070000277800801F78003E0078005D
:100DB00087FD0700002778004F0078002000B00072
:100DC00083FD0700000006001C000000C4454D0024
:100DD00049540000002778000027780030012000E7
:100DE000D2FD07002BFD070000277800100120002E
:100DF000CEFD07003E007000D9FD07000000B000E6
:100E00003E0078001E00320037FF07001000780017
:100E10000000B0003E0078000E003200002778008D
:100E200080BB200030FF070069FD07000027780025
:100E3000A0002000BDFD07000000B0003E007800CB
:100E40000300320000277800E00220000100370094
:100E500000000600002778000000B0003E00780087
:100E600007003200A1FF07002008B00053FD070073
:100E700094FD07000000B0003E007800F9FF32004A
:100E8000002778000000280090FF07000027780066
:100E9000801F78003E00780000277800100078005E
:100EA000801F78003E00780049FD07000027780089
:100EB000E0202000100078000027780000202000AB
:100EC0003E0060000000B0003E00780003003200E9
:100ED0000027780000002000050037000027780078
:100EE000002120003AFD070000277800F0FF2F00C6
:100EF0000000B0003E007800ECFF320000277800D0
:100F00004F007800002778004F00780030FD070080
:100F100000000600A6000000C45052004740000038
:100F200079FF0700811F7800821F7800BE007800DB
:100F30001000A7001500370002FC2F00028160009E
:100F40001010E10011003A00100190001E10E100A5
:100F50000E003A004000B000E103B2000080400003
:100F6000C108DE00008040000001EB000000A60088
:100F7000B0007800304178000000A600B000780092
:100F8000020F7800010078000500370022032000DE
:100F90001E0978001181BA00020F78001100BA0012
:100FA0004F017800CF007800000006004C000000E0
:100FB000C45052004721000053FF0700811F7800F2
:100FC000821F7800BE00780002FC2F0002816000C2
:100FD0001010E10003003A00100190001E10E10023
:100FE000060032001000A6002800070002FC2F00B7
:100FF000029860001E107800110007004000B00049
:10100000E103B20000804000C108DE000080400023
:1010100062074700BE0078003E0178000000A6008D
:1010200001187800025878000000A6000118780026
:101030003E0078004F017800CF00780000000600E5
:10104000811F7800821F7800831F7800841F78003A
:10105000B00078002203200030097800F30020005F
:101060001101BA003182BA000218780004587800E1
:101070001101BA003182BA000458780002187800D1
:101080008301E900F6FF31002C003700811F780052
:10109000821F7800831F7800841F780021042000BD
:1010A000020E2000911F780091087100B0007800B6
:1010B000227620000119780010097800120424001B
:1010C000023B880052052000323B8800A20A200023
:1010D000323B880061E7A80000000000000000002B
:1010E00012002400023B880022032000300978000F
:1010F000F300200030017800304278008208BB0005
:101100008498BB0030427800300178008208BB0030
:101110008498BB008301E900F6FF310052052000EE
:10112000323B8800A20A2000323B880061E7A80019
:1011300000000000000000004200F9004006B1007D
:101140004F027800CF0178004F017800CF0078007F
:1011500000000600D4000000C4505200472C0000DC
:1011600001FF07004BFC07004AFC0700002778003E
:10117000000020000027780020002000A3FC0700CA
:1011800007FF07008CFF0700000006001C0000009E
:10119000C445450050400000811F78002103200015
:1011A000BE0878001000BA00CF00780000000600EA
:1011B00012000000C445450050210000811F780046
:1011C00062A7B7009E007800213B880041042400FC
:1011D000013B88000500FC0051052000313B8800E0
:1011E000A10A2000313B880061E7A8000000000050
:1011F0000000000061E7AF00FEFF37002103200080
:10120000BE0878003E08BB0041002400013B880076
:101210000500FC0051052000313B8800A10A200098
:10122000313B880061E7A8000000000000000000DA
:1012300061E7AF00FEFF37003E007800CF00780086
:10124000000006004A000000CB7370005F73790055
:101250006E63700072672100ABFE07001000A600ED
:101260008AFF07001000A0003E0078000000060082
:1012700060000000C4484500524500005EFE0700C3
:1012800010007800000006000C000000C53E480079
:101290004552450058FE07004DFC070000000600BF
:1012A0000C000000C2432C00F4FF07000027780068
:1012B0001000B000F7FF07004AFC0700000006001E
:1012C00010000000C12C0000ECFF07000027780090
:1012D0002000B000EFFF07003DFC07000000060003
:1012E00010000000CA7370005F636F006D706900CA
:1012F0006C650000E7FB0700E6FB070008FF07003E
:10130000801F78003E007800002778003E006800CB
:10131000002778007FB8970000277800F0032000AE
:101320003E0060001000B000002778003000200070
:10133000C8FC0700D0FB070069FC07003E00100056
:101340004100DD0031FC0700002778004F007800E5
:1013500000277800000420003E0060000000B0007C
:101360003E007800310032007FFE07000027780041
:1013700000002000002778002000200023FC070048
:1013800034FC0700C3FB070000277800F0FF2F00A4
:1013900066FC07000000B0003E0078000D0032003F
:1013A000801F78003E0078003E007800002778001B
:1013B00070002000002778004F0078004180DE0098
:1013C00000277800000028003E00700064FF07003E
:1013D0001500370064FE0700002778000000200099
:1013E000002778002000200008FC070007FC070009
:1013F000801F78003E007800002778002000200041
:10140000002778004F00780055FF0700801F780004
:101410003E007800002778000000200000277800B8
:101420004F0078004EFF07001700370099FB0700B8
:1014300098FB0700BAFE070049FF07000027780065
:10144000000020000027780020002000EFFB0700AC
:1014500090FB07008FFB0700B1FE070019FC070097
:1014600085FB070000277800600020002FFC0700A4
:101470003E0060000000B0003E007800EBFF32004C
:101480003E0078003E00780000000600E600000004
:101490004249460000277800000B20000027780012
:1014A000000020002EFF07000027780080072000A2
:1014B00000277800E003200029FF070000277800BC
:1014C0002003200000277800F0FF2F0024FF0700F2
:1014D00025FE07000000060026000000C77370000C
:1014E0005F73610075740000801F78003E00780013
:1014F000801F78003E00780066FB070065FB070050
:10150000002778000000200000277800200020003D
:10151000D0FB070082FE07003E007800002778001D
:101520004F007800002778004F00780000277800EF
:101530005000200065FB07000027780050002000C5
:1015400062FB0700C3FB0700801F78003E007800A5
:1015500000277800F0002000BDFC0700002778007D
:101560004F00780000277800F0FF2F00B8FC07003C
:101570003E004000002778004000200063FB070089
:10158000002778004000200060FB0700002778005B
:10159000000020000027780020002000ADFB07009D
:1015A00085FE0700000006008E00000044454C0048
:1015B00053450000002778007003200000277800C2
:1015C000F0FF2F00E6FE0700E7FD0700C6FF07005B
:1015D000E5FD070000000600180000004454480024
:1015E000454E0000E0FD0700BFFF070000000600B9
:1015F0000C000000444341005345000000277800E0
:10160000000020000027780000277800000020005C
:1016100000277800601B200036FF0700000006004E
:1016200018000000424F460000277800000020000C
:1016300000277800A01C20002EFF0700002778005C
:1016400000002000002778004029200029FF070023
:1016500090FF0700000006001C00000045454E00FA
:10166000444F4600D3FF0700000006000A000000B8
:1016700047454E004443410053450000A8FD070084
:101680004180DE0034FB07000000B0003E0078001F
:101690002500320000277800300020000BFB0700F7
:1016A000002778003000200008FB07003E00700093
:1016B0000000B0003E00780008003200801F780073
:1016C0003E007800A8FD070087FF0700002778008C
:1016D0004F0078001000B100020037003E00780093
:1016E0003E0078000027780076FB07000000B0007D
:1016F0003E007800E7FF32003E00780000277800C7
:101700000000200000277800001C2000F9FE0700E0
:10171000002778000000200000277800E01020005B
:10172000F4FE07000200370000277800F0FF2F00CA
:1017300000000600640000004542450047494E0095
:1017400089FD0700000006000A00000045554E0014
:1017500054494C004FFF070000277800400020004C
:10176000EAFA07000027780040002000E7FA0700A7
:101770005DFF070000000600180000004557480004
:10178000494C450043FF0700000006000A00000026
:1017900046524500504541005400000085FF0700B7
:1017A0000027780040002000D8FA070000277800C2
:1017B00040002000D5FA07004BFF0700000006009C
:1017C0001A00000042444F0000277800000020006B
:1017D0000027780080132000C6FE070062FD070086
:1017E000002778000000200000277800601B200000
:1017F000C0FE0700002778000000200000277800C6
:10180000601B2000BBFE0700000006002600000051
:10181000452B4C004F4F500000277800000020005F
:1018200000277800001C2000B2FE07000027780087
:101830000000200000277800C01F2000ADFE070038
:10184000002778000000200000277800001C2000FE
:10185000A8FE07000027780000002000002778007D
:1018600060142000A3FE070000277800000020007D
:1018700000277800601420009EFE070000277800F3
:1018800000002000002778008028200099FE070033
:10189000002778000000200000277800C02A2000E0
:1018A00094FE0700ABFF070000277800000020002F
:1018B00000277800E01020008EFE07000027780047
:1018C0000000200000277800E010200089FE0700BB
:1018D0000000060064000000C74C49005445520057
:1018E000414C000000277800800720000027780086
:1018F000007022001AFE070000277800801F780081
:101900003E0078000027780040FF2F00D0FB070042
:101910000002B000002778004F0078000027780010
:1019200040002000CAFB07000DFE07004AFE07002A
:101930000000060030000000444C4F004F500000F3
:101940000027780010002000E6FF0700B2FF070024
:101950000000060010000000814900000027780008
:101960007FB89700000006000A000000814A0000CE
:10197000002778005FB89700000006000A0000000A
:10198000814B0000002778003FB897000000060058
:101990000A000000854C45004156450000277800AC
:1019A0004F0078004F007800801F7800801F78007B
:1019B0003E00780000000600140000008445580036
:1019C000495400000000060008000000C243520015
:1019D00000277800D0002000FEFC070000277800D8
:1019E000A0002000FBFC0700000006001200000021
:1019F000C44245004C4C00000027780070002000D5
:101A0000F4FC0700000006000E000000C553500063
:101A1000414345000027780000022000EDFC07004C
:101A2000000006000E000000C65350004143450070
:101A30005300000048FA07000000B0003E007800A4
:101A400008003200F3FF07001000B1000027780003
:101A50009CFA07000000B0003E007800F9FF320059
:101A60003E0078000000060022000000C454590027
:101A7000504500000027780099FA07000000B000E8
:101A80003E0078002F0032001000B100801F780067
:101A90003E0078000027780048FA07000027780009
:101AA000F00F20003E0060000027780085FA070054
:101AB000F8F9070000277800300020009BFA0700A3
:101AC0003E0070000000B0003E00780009003200C7
:101AD0003E007800002778004F0078003E00780034
:101AE0000027780000002000801F78003E0078006A
:101AF0000B0037000027780000277800D000200076
:101B00008AFA07000000B0003E00780003003200AF
:101B10003E007800AEFF070001003700ADFC070073
:101B20001000B000002778004F00780000277800F0
:101B300064FA07000000B0003E007800D2FF3200D7
:101B400069003700002778004F80DE000000B000F9
:101B50003E00780064003200801F78003E0078006C
:101B6000CCF90700CBF90700EDFC0700002778004F
:101B70004F0078000000EA00002778000000B00065
:101B80003E00780014003200801F78003E0078008C
:101B90000027780080FF2F002DFB0700002778002A
:101BA00000277800D000200060FA07000000B00095
:101BB0003E007800030032003E00780084FF0700FA
:101BC0000100370083FC0700002778004F007800F1
:101BD0001000B10002003700A7F907003E007800AE
:101BE00000277800801F78003E0078000000B000D9
:101BF0003E007800110032000027780000277800AE
:101C0000D000200049FA07000000B0003E00780034
:101C1000030032003E0078006DFF0700010037002E
:101C20006CFC0700002778004F0078001000B1001E
:101C3000801F78003E007800010037003E007800E9
:101C400000277800000020000027780020002000F6
:101C5000EEF907008FF907008EF90700B0FC0700C6
:101C6000002778004F007800002778000000B000BF
:101C70003E00780014003200801F78003E0078009B
:101C80000027780000277800F00F20003E00600059
:101C90000027780000277800D000200023FA0700F2
:101CA0000000B0003E007800030032003E007800E3
:101CB00047FF07000100370046FC070000277800B7
:101CC0004F0078001000B10000277800FDF90700F0
:101CD0000000B0003E007800A7FF32003E00780010
:101CE0003E0078003E0078003E0078003E0078001C
:101CF0000000060046010000C5434F00554E540049
:101D0000002778001000B0005BF90700ABF907006E
:101D100000277800F00F20003E0060000000060061
:101D200016000000C92D5400524149004C494E0094
:101D30004700000000277800E9F907000027780035
:101D40003000200061F907000027780030002000F3
:101D50005EF907001000B1003E00400097F907004F
:101D60000027780000022000F0F907003E00600024
:101D70000000B0003E007800020032001000B10008
:101D8000ECFF37000000060034000000C3424900A9
:101D90004E0000000027780020002000B0FB070064
:101DA0008BF907000000060010000000C54F43003B
:101DB00054414C000027780080002000A8FB070059
:101DC00083F907000000060010000000C74445002A
:101DD00043494D00414C000000277800A00020003E
:101DE0009FFB07007AF907000000060012000000C0
:101DF000C34845005800000000277800000120007B
:101E000097FB070072F907000000060010000000B1
:101E1000C7434F004E564500525400001000B0001A
:101E200000277800000020001AF9070063F9070076
:101E30000027780000277800B0022000BBF90700D7
:101E40000000B0003E007800070032003E0078003D
:101E5000801F78003E0078001000B0000027780056
:101E60004F0078000C00370000277800D0022000D7
:101E7000AEF907000000B0003E0078000600320016
:101E8000801F78003E0078001000B0000027780026
:101E90004F0078001000B100801F78003E007800ED
:101EA0000027780045F907000003B10000277800FB
:101EB0004F80DE000000B0003E00780004003200D9
:101EC0003E00780000277800F0FF2F003500370033
:101ED00000277800002778009000200099F907007B
:101EE0000000B0003E007800060032007000B10033
:101EF0000027780000277800A000200085F907005F
:101F00000200370000277800000020000000B00029
:101F10003E007800040032003E0078000027780080
:101F2000F0FF2F001F003700002778004CFB070050
:101F30001000780077F907000000B0003E0078003C
:101F400015003200801F78003E007800801F780066
:101F50003E00780042FB07001000780086F9070079
:101F6000002778004F0078001000B00000277800AC
:101F70004F007800C0F80700801F78003E0078000E
:101F80003E004000002778004F00780000277800CE
:101F900000002000030037003E0078000027780092
:101FA000F0FF2F000000B0003E007800BCFF3200C0
:101FB000002778004F0078000000B0003E00780055
:101FC00005003200801F78003E0078000000EA0023
:101FD000002778004F00780000000600E8000000AD
:101FE000C23C23000027780000002000B2FA07005E
:101FF000FCF8070000277800801F78003E0078007A
:102000004F80DE00002778004F007800ECF90700D1
:10201000000006001C000000C4484F004C440000B3
:10202000A5FA0700002778001000B000002778000C
:102030001000B0000027780030002000A3F807004F
:10204000DEF8070000277800F00F20003E00600057
:1020500000277800E0052000D2F907004BFA0700BE
:1020600000277800D5F8070000277800F00F20003F
:102070003E0060001000B00000277800E00520005E
:10208000C8F9070083F80700D6F807001000B00071
:10209000D4F807000000060042000000C123000041
:1020A000EFFA07001000780040F9070072F8070007
:1020B0000003B0000027780000277800900320007C
:1020C00020F9070000277800700020003E00600023
:1020D0003E004000D2FF0700000006002200000082
:1020E000C2235300EEFF0700002778001CF9070009
:1020F0000000B0003E007800FAFF32000000060049
:1021000012000000C4534900474E000061F8070068
:102110000000B0003E007800030032000027780085
:10212000D0022000BEFF07000000060016000000DD
:10213000C2233E003E0078003E0078005EFA0700B1
:10214000EFFE0700000006000E000000C12E000098
:10215000A4FF07000027780000022000B0FF07005E
:10216000E0FF0700E9FF0700F2FF070041FE07005C
:102170000000060016000000C13F000010007800BB
:10218000F3FF0700000006000A000000C2552E0001
:10219000002778000000200092FF07000027780049
:1021A000000220009EFF07003E00780032F8070082
:1021B000CCFF0700DFFF07002EFE0700000006002F
:1021C0001C000000C4574F0052440000801F7800DC
:1021D0003E00780031FA0700002778000000200058
:1021E0002CF807007FF80700002778000000200087
:1021F0008FFA070076F8070000277800000020001B
:1022000091FA070072F8070044FA070010007800FE
:1022100048FA0700100078003E00400000277800D0
:10222000801F78003E0078001000B0000027780082
:10223000100020003FFA0700B5F9070000277800DA
:102240004F0078005DF8070000277800F00F2000AD
:102250003E00600000277800801F78003E00780074
:10226000002778003000200018F8070000277800C9
:1022700052F807003E0040001000B00059F8070077
:10228000002778004F007800002778008DF80700BD
:1022900000F807000027780030002000A3F80700AE
:1022A0003E0070000000B0003E0078000A003200DE
:1022B0003E00780000277800F0FF2F00002778000C
:1022C0005BFA070042F80700002778005EFA070073
:1022D0003FF807002E00370000277800002778001D
:1022E000D000200091F807000000B0003E00780008
:1022F000070032003E00780000277800F0FF2F0032
:10230000002778004AFA070031F80700200037005C
:1023100000277800801F78003E00780000277800B2
:102320009000200081F80700002778007FB8970010
:1023300000277800000220007CF807003E007000B3
:10234000002778004F007800002778007FB89700BA
:1023500076F807003E0070000000B0003E007800F4
:102360000300320000277800F0FF2F00080037003C
:10237000002778001000200000277800300020009F
:10238000D2F7070051F9070000277800000020006D
:102390000000B0003E007800A0FF32003E00780050
:1023A000002778004F0078003E007800000006000B
:1023B000F8000000C127000000277800000220007C
:1023C00082FF070000277800FCF707000000B0003C
:1023D0003E007800CE003200801F78003E0078007A
:1023E000F2F9070000277800801F78003E0078008F
:1023F0002000B00010007800002778004F0078001F
:1024000010007800002778007FB897000027780038
:1024100000277800E9F707003E0040001000B000F8
:102420000027780040002000A8F707000027780068
:1024300040002000A5F7070096F7070095F7070072
:10244000B7FA070000277800F0F32F003E00600085
:10245000002778004F0078008EF7070000277800EB
:10246000F00F20003E0060008AF70700D3F7070056
:1024700000277800F00F20003E0060002BF80700D6
:102480000000B0003E007800350032001000B000BF
:1024900000277800600020008CF707007DF7070018
:1024A00028F807000000B0003E0078002900320044
:1024B00078F707000027780080FF2F00E4F8070076
:1024C00074F70700BDF7070018F807000000B00018
:1024D0003E0078001C0032001000B0000027780099
:1024E0006000200079F707006AF7070015F8070079
:1024F0000000B0003E007800100032000027780095
:102500003000200071F7070062F70700ABF7070003
:1025100006F807000000B0003E007800040032001A
:102520001000B00000277800F0FF2F0002003700F5
:102530000027780000002000020037000027780004
:10254000F0FF2F0002003700002778000000200075
:102550000200370000277800F0FF2F00020037004C
:102560000027780000002000801F78003E007800DF
:10257000801F78003E0078003E0078003E00780022
:10258000002778004F007800002778004F0078007F
:102590000000B0003E0078001F00320000277800E5
:1025A0004000200049F707003AF70700E5F7070069
:1025B0000000B0003E0078000F003200801F78005D
:1025C0003E007800002778000000200000277800F7
:1025D000200020008DF707002EF707002DF70700D9
:1025E0004FFA0700002778004F0078000027780096
:1025F00000002000070037003E0078003E00780011
:102600003E0078003E0078003E0078000027780009
:10261000F0FF2F003A0037003E0078003E007800BF
:102620003E007800801F78003E007800801F780010
:102630003E00780017F7070016F70700002778001C
:1026400000002000002778002000200081F707000C
:1026500033FA07000FF707000EF707003E0070007F
:102660000000B0003E0078001700320079F7070044
:10267000002778004F007800002778004F0078008E
:10268000002778004000200010F70700002778009E
:10269000400020000DF70700FEF60700FDF60700DA
:1026A0001FFA070000277800F0F32F003E006000BB
:1026B000002778006000200004F70700002778005A
:1026C000000020000E003700002778004F0078003F
:1026D000002778004F0078003E0078003E00780028
:1026E0003E0078003E0078003E0078000027780029
:1026F0003E0068000027780000277800F0FF2F00D8
:102700000000B0003E00780053FF320003003700A5
:10271000002778003E0068000027780000000600CF
:10272000B8010000C44649004E44000022FF0700E3
:10273000D8F60700D7F607003E0070000000B00092
:102740003E00780015003200D2F60700D1F60700EF
:10275000F3F90700801F78003E007800002778001A
:102760003E006800002778004F00780000277800BE
:10277000F00320003E0060001000B0000027780049
:1027800030002000B3F70700BBF6070054F707003E
:102790003E0010004100DD001CF7070000000600AD
:1027A00040000000415B000000277800000020008E
:1027B00031F9070006F70700000006000E000000D0
:1027C000C15D000000277800F0FF2F002AF9070004
:1027D000FFF60700000006000E000000C13A0000EE
:1027E000002778000002200078FE07005EF907004D
:1027F000002778000000200000277800200020003B
:1028000002F70700E9F8070000277800801F78002A
:102810003E0078002000B00010007800002778000B
:102820007FB89700100078000AF707004CFA0700FD
:102830004DF90700002778007FB89700E4F60700FD
:10284000002778004F0078002000B000E0F6070075
:1028500000277800D9F6070000277800F003200051
:102860003E0060001000B000801F78003E0078003D
:10287000002778002000B000D0F60700002778007D
:10288000F00F20003E00600082F607001000B0004C
:10289000CAF607000027780080002000ECF7070048
:1028A000002778007FB897001000B100002778005B
:1028B000000C20003E0070003E00400028FA070097
:1028C0003000B000002778004F0078003000B100E1
:1028D0000027780002F707000000B0003E007800F3
:1028E00016003200801F78003E0078000027780034
:1028F0002000B000B1F6070000277800F00F20009C
:102900003E00600063F607001000B000ABF6070061
:102910000027780080002000CDF70700002778000E
:102920003000200069F60700A4F6070000277800B1
:10293000F00F20003E006000DFFF37003E0078000F
:102940003E00780000277800F0FF2F00CAF807004B
:102950009FF60700F2F807007EF807009CF60700D4
:1029600000000600C6000000413B00000027780080
:10297000600020000027780000002000F8F9070020
:1029800035FA07000027780000002000BAF8070099
:102990008FF60700E2F807006EF8070010007800D5
:1029A0003E0010000000B0003E0078000E00320033
:1029B0000027780030002000B5F8070084F60700F3
:1029C00056F8070010007800B1F807002000B000AA
:1029D0007FF6070057F8070010007800ACF80700F2
:1029E0004000B0007AF60700000006004400000036
:1029F000C87370005F746100636865000027780029
:102A00004F007800002778004F00780000277800FA
:102A1000300020002DF6070000277800801F780086
:102A20003E0078008000B00069F6070000277800BB
:102A30004F007800A000B00065F607000000060017
:102A40006E000000C6544100434845003A000000B3
:102A500063FF070009FA0700A2FB070000277800C0
:102A60000000200018FA070000277800000020006E
:102A700015FA0700002778000000200012FA07006E
:102A800000277800000020000FFA070000277800D8
:102A9000000020000CFA070000277800000020004A
:102AA00009FA0700002778000000200000277800BE
:102AB000804F21000FFA0700000006003E000000D2
:102AC000C9545F0045584500435554004500000077
:102AD00000277800801F78003E007800A000B0003A
:102AE00010007800002778004F0078008000B000C8
:102AF00010007800801F78003E007800801F78006A
:102B00003E0078000000060026000000C8545F0068
:102B1000414A4F005554450065F8070000277800EA
:102B2000801F78003E0078001000780000277800B1
:102B3000F0FF2F00002778007FB8970024F60700E9
:102B4000801F78003E00780024F8070000277800F6
:102B50001000780000F607000000B0003E0078008A
:102B6000350032000027780030002000D7F507003C
:102B7000C8F507006DF607000000B0003E007800C1
:102B8000070032003E0078003E0078003E007800EA
:102B90003E00780000277800F0FF2F002500370066
:102BA00000277800100078000027780050002000EF
:102BB000C6F5070051F607000000B0003E0078009F
:102BC000140032000027780030002000BFF5070015
:102BD0004000B000FEF50700801F78003E0078003E
:102BE00000277800002778004F007800F8F50700EC
:102BF00000277800F0FF2F00A6F507002000B000A6
:102C0000F3F50700F2F5070000277800F0FF2F002A
:102C100008003700801F78003E0078003E007800F2
:102C2000002778004F0078004000B00000277800AF
:102C30000000200013003700801F78003E0078005D
:102C400000277800002778004F007800E0F50700A3
:102C500000277800F0FF2F008EF507002000B0005D
:102C6000DBF50700002778000000200089F5070049
:102C70004000B000D6F50700D5F507000027780022
:102C8000F0FF2F000000B0003E007800AFFF3200E0
:102C9000002778004F007800002778004F00780068
:102CA000CBF5070000000600D0000000C8545F000C
:102CB0004143540049564500801F78003E0078008B
:102CC0000027780010002000ADF6070000277800EC
:102CD00000002200B3F60700002778004F007800BC
:102CE0006000B000BAF507000000060022000000F6
:102CF000C9545F0050455200494F44004500000050
:102D0000801F78003E007800002778001000200027
:102D10009BF607000027780000002200A1F60700BC
:102D2000002778000000EA00002778007FB89700AD
:102D30006000B000A6F507004180DE00A1F70700A3
:102D4000100078003E00400000277800F0FF2700C8
:102D50003E006000002778004F0078002000B0009F
:102D60009BF50700000006003E000000C8545F000D
:102D7000524554004952450077F507000000B00065
:102D80003E0078003D003200C9F7070000277800B8
:102D9000801F78003E00780010007800002778003F
:102DA000F0FF2F00002778007FB8970088F5070014
:102DB000801F78003E00780088F7070035F507008F
:102DC00034F5070010007800D8F507000000B000C7
:102DD0003E00780015003200801F78003E00780029
:102DE00000277800000020002AF507006000B000EE
:102DF00077F50700002778004000B0001000780049
:102E0000002778004F00780071F507000027780050
:102E1000000020001FF507004000B0006CF507001F
:102E200000277800F0FF2F000B003700100078001B
:102E300049F507000000B0003E00780004003200B1
:102E40004000B0000027780000002000020037009A
:102E500000277800F0FF2F000000B0003E0078004F
:102E6000D6FF32003E007800002778004F0078003F
:102E7000002778004F00780055F507000000060095
:102E80008C000000C57370005F2E6700002778007B
:102E90004F007800002778004F007800FDF407000D
:102EA000FCF407001EF8070000277800F00F200050
:102EB0003E006000801F78003E0078003E007800F1
:102EC000F4F40700F3F40700002778000000200066
:102ED000002778007FB897001000B0000027780026
:102EE00030002000DBF50700E3F407007CF5070065
:102EF0003E0010004100DD0044F507000027780087
:102F00004F007800DCF40700801F78003E00780056
:102F1000D9F40700801F78003E0078000000EA0026
:102F2000D4FA070000000600E0000000C5544C0081
:102F30004953540029F707001000780006F50700F0
:102F40000000B0003E0078007000320000277800DA
:102F5000A000B00010007800CEF407008000B000A0
:102F6000100078000027780000002000002778007B
:102F70002000200037F50700C6F40700C5F407005D
:102F8000E7F707003E007800002778008007200060
:102F900066F507000000B0003E007800F1FF320047
:102FA0000027780000002000002778002000200083
:102FB00028F50700B7F40700B6F40700D8F70700B4
:102FC000801F78003E0078003E00780000277800DF
:102FD0004F007800002778000027780000082000C4
:102FE0003E0060000000B0003E00780009003200A2
:102FF00000277800F00320003E0060000000EA0097
:103000009CFA070083FA070000277800F0FF2F00E2
:1030100002003700002778003E0068000000B00082
:103020003E007800DEFF32000DF707001000780048
:10303000801F78003E00780067FB070093FF0700C1
:103040000B707200696F720069746500203A20008D
:1030500000277800100078004DFC07002000B00029
:10306000002778004000B0001000780000277800AA
:103070004F80DE000000B0003E0078000B00320000
:1030800082FF07000D70650072696F00646971004E
:10309000756520003A2078000000EA002CFC07004B
:1030A0007AFF0700026D7300110037003E007800C0
:1030B00000277800100078004F80DE000000B0008C
:1030C0003E0078000600320070FF070009494E00FC
:1030D0004143540049564500206520000400370054
:1030E0006AFF070007414300544956004520450048
:1030F000002778004F007800D9F60700B4F40700E5
:1031000033FA07002000B0008BFF370000000600F4
:10311000F400000047434F004D5049004C4500006B
:10312000A5FC07005BF407005AF407003E0070009E
:103130000000B0003E007800090032004EF40700A5
:10314000E8F90700E7F907000027780000002000F1
:10315000002778002097200066F80700100037004D
:103160003E0078003E007800002778003000200004
:10317000C7F6070096F4070068F60700100078000D
:10318000C3F607002000B00091F4070069F60700BD
:1031900010007800BEF607004000B0008CF4070075
:1031A000000006004A000000495B43004F4D5000FC
:1031B000494C45005D0000007FFC070035F4070026
:1031C00034F407003E0070000000B0003E007800BC
:1031D0000200320047F80700100037003E00780078
:1031E0003E0078000027780030002000A8F6070095
:1031F00077F4070049F6070010007800A4F60700EE
:103200002000B00072F407004AF6070010007800B2
:103210009FF607004000B0006DF4070000000600B4
:103220003E000000C7455800454355005445000086
:10323000801F78003E007800801F78003E007800F4
:103240000000060012000000C122000000277800E4
:103250004000200088F60700ADF50700C2F6070021
:1032600000277800F00F20000027780000002000E1
:103270000000060018000000422E220000277800FF
:1032800000002000002778002074210019F80700B2
:10329000EEFF0700000006001200000001280000F9
:1032A000002778002000200073F6070098F507003B
:1032B000000006000E000000C22E530098F6070022
:1032C00025F407000000B0003E0078001C0032002A
:1032D0000027780000002000801F78003E00780062
:1032E000002778001000B000002778007FB8970012
:1032F0003E001000F5F3070095FB0700002778005B
:103300004F0078001000B00000277800801F780080
:103310003E007800DFF307007EF4070090F407001A
:103320000000B0003E007800EDFF3200002778007A
:103330004F0078003E0078003E007800060037001D
:10334000D2FE07000C5069006C65200076696400AD
:1033500065202100202078000000060054000000B5
:1033600049494D004D454400494154004500000085
:103370000EF6070000277800801F78003E007800D6
:103380002000B00010007800002778004F0078007F
:1033900010007800BFF30700BEF30700E0F6070057
:1033A00000277800F0F72F003E006000002778002B
:1033B00040002000D5F307000027780040002000DF
:1033C000D2F30700FCF607000000060038000000FA
:1033D000464449005245430054000000F3F50700FD
:1033E00000277800801F78003E0078002000B000A1
:1033F00010007800002778004F0078001000780057
:10340000A4F30700A3F30700C5F607000027780020
:10341000F0FB2F003E0060000027780040002000F5
:10342000BAF307000027780040002000B7F3070038
:10343000E1F607000000060036000000C5414C0020
:103440004C4F5400002778000000B0003E00780088
:103450000500320000277800000020009AF70700DE
:103460001000B100F7FF37003E00780000000600B2
:103470001C000000C44C4F004144000004F607004B
:10348000100078000000B0003E007800020032001A
:103490003E007800F50137000CF6070010007800B8
:1034A000801F78003E007800002778001000200080
:1034B00006F60700C6F3070098F50700100078002D
:1034C000801F78003E0078009AF507001000780011
:1034D000801F78003E007800D5F5070010007800C6
:1034E000801F78003E007800D7F5070010007800B4
:1034F000801F78003E00780088F50700B4F30700CD
:1035000000277800000020008AF50700B0F30700CC
:10351000D9F507001000780000277800F0F30700C5
:103520000000B0003E007800B600320000277800AE
:103530002000200003F407000000B0003E007800E7
:10354000A100320000277800200220001FFB0700A6
:10355000EBF9070000277800300020005BF307003C
:1035600000277800F00F2000E4F3070049F307007C
:10357000DBF307003E0060000000B0003E00780072
:103580002C003200801F78003E007800801F7800F9
:103590003E00780038F307006FF307000000B0002A
:1035A0003E007800170032000027780000277800DE
:1035B00000102000D1F307000000B0003E007800AA
:1035C00008003200002778007FB897007BF30700DF
:1035D00000277800800020009DF407003E00400096
:1035E00007003700002778007FB8970073F30700C3
:1035F00021F30700DAF6070000277800000020001A
:1036000003003700002778007FB897006BF30700AE
:1036100019F307001000B000002778004F00780071
:103620001000B000002778004F0078001000B100B3
:10363000C8FF37003E00780060F3070000277800DD
:103640000027780020022000B8F307000000B00037
:103650003E0078002A0032003E007800801F78008B
:103660003E0078003CF307000000B0003E00780008
:10367000040032000027780000002000FEF207005E
:10368000B7F6070003F3070002F3070024F607006C
:103690000027780000F02F003E006000002778002F
:1036A0004F0078003E0040000027780040002000D6
:1036B00006F30700002778004000200003F307000E
:1036C0003DF607006CF50700100078000027780031
:1036D0003000200095F307000000B0003E007800A5
:1036E000020032003E0078003E007800002778009B
:1036F0004000200060F507008DF40700310037001E
:1037000051F50700100078000000B0003E0078007E
:10371000030032003E00780000277800D00020002F
:10372000DCF2070000277800F00F200073F3070099
:103730000000B0003E00780021003200801F7800B9
:103740003E007800CCF2070003F307000000B00051
:103750003E0078001500320000277800002778002E
:103760000010200065F307000000B0003E00780064
:1037700007003200002778004F007800002778000B
:103780008000200032F407003E00400006003700B1
:10379000002778004F007800B7F2070070F60700A6
:1037A0000027780000002000020037000027780082
:1037B0004F007800B0F207001000B00001003700A1
:1037C0003E0078000E00370000277800000220003D
:1037D0007EFA070010007800002778001090220081
:1037E00052F307000000B0003E00780004003200F1
:1037F00000277800200020001FF507004CF4070088
:10380000EB0037003E007800EBFA0700A1F207005A
:10381000A0F207003E0070000000B0003E007800FB
:103820005F00320014F50700100078000000B000BF
:103830003E0078002400320096F2070095F207005F
:10384000B7F507008CF207003E00780000277800EB
:10385000000820003E0060000000B0003E0078003C
:1038600002003200A3F607001600370089F20700B5
:1038700088F20700AAF50700801F78003E00780054
:10388000002778003E006800002778004F0078008D
:1038900000277800F00320003E0060001000B00018
:1038A00000277800300020006AF3070072F207005A
:1038B0000BF307003E0010004100DD00D3F20700CB
:1038C0005BFE07003500370072F2070071F2070057
:1038D00093F5070068F207003E00780000277800A3
:1038E000000C20003E00600000277800000420004B
:1038F0000EF307000000B0003E0078001100320017
:103900003E0078003E00780000277800200020006C
:10391000DFF40700AEF2070080F407001000780023
:10392000DBF407002000B000A9F2070081F40700D3
:1039300010007800D6F407004000B000A4F20700A1
:103940001600370053F2070052F2070074F5070023
:10395000801F78003E007800002778003E00680055
:10396000002778004F00780000277800F00320003F
:103970003E0060001000B0000027780030002000FA
:1039800034F307003CF20700D5F207003E001000B8
:103990004100DD009DF2070025FE0700840037008E
:1039A0003E0078003DF407000027780083F207000E
:1039B0000000B0003E0078007B00320035F20700C6
:1039C00034F2070015F9070038F207003E007800CE
:1039D00036F207003E0078000027780077F20700F3
:1039E0000027780010022000CAF207000000B00093
:1039F0003E007800080032003E0078009EF4070088
:103A0000100078000000B0003E0078000100320095
:103A1000B4F70700630037000027780067F207005B
:103A20000027780000277800B0022000BFF20700CE
:103A300011F2070000277800D0022000BBF2070037
:103A40003E00700013F207001000B0005BF20700A8
:103A50000027780010022000AEF207003E00600050
:103A60000000B0003E0078003E00320009F207007E
:103A70000000B0003E007800370032004FF207002F
:103A80007DF40700100078000000B0003E007800D0
:103A900027003200801F78003E0078000027780061
:103AA000002778000040200094F207000000B000DA
:103AB0003E0078000E003200002778004000200011
:103AC00063F30700002778004F0078000027780094
:103AD000D002200095F20700002778001000200097
:103AE0003E006000000BB000E3F107000E0037005D
:103AF0007CF70700002778000004200000277800EA
:103B00004F00780000277800D002200087F20700DD
:103B100000277800000320003E0060003E001000F7
:103B200000277800E00320008DF50700090037002A
:103B300000277800B00220007CF207000000B000EF
:103B40003E007800020032003E00400001003700D5
:103B50003E001000020037003E0078003E00780072
:103B6000100037003E0078003E0078000027780003
:103B70001000200046F4070015F20700E7F30700E5
:103B80001000780042F407002000B00010F2070097
:103B9000E8F30700100078003DF407004000B00093
:103BA0000BF20700020037003E0078003E0078006C
:103BB00025F407001000780035F4070010007800A5
:103BC0003E0070000000B0003E00780050FE320061
:103BD00053F407004F80DE000000B0003E00780084
:103BE0000E003200002778004000200028F4070073
:103BF000F7F10700C9F307001000780024F407006C
:103C00002000B000F2F10700CAF3070010007800AE
:103C10001FF407004000B000EDF107000027780016
:103C20004F00780008F40700E9F10700002778004A
:103C30004F007800FEF30700E5F107000027780049
:103C40004F007800BBF30700E1F107000027780080
:103C50004F007800B1F30700DDF10700002778007E
:103C60004F00780019F40700D9F1070000000600A2
:103C700000040000C64352004541540045000000C6
:103C80007EF5070017F7070037F40700C1F30700B8
:103C900000277800801F78003E007800CCF10700F4
:103CA000002778004F0078002000B000C8F107001E
:103CB000002778004000200000277800F0FF2F0048
:103CC00027F5070000277800000020000027780073
:103CD000F007200022F507005FF50700000006004E
:103CE00038000000C87370005F646F0065733E00A9
:103CF000A8F3070000277800801F78003E007800B6
:103D00002000B00010007800002778004F007800F5
:103D100010007800002778000000200000277800BD
:103D20004F007800002778004000200067F107006E
:103D3000002778004000200064F107000027780089
:103D4000000020000027780020002000AFF10700CD
:103D500099F4070000277800400020000027780031
:103D60004F007800002778004000200067F107002E
:103D7000002778004000200064F107008EF407005F
:103D800035F507000027780000002000BAF307008F
:103D90008FF10700000006009400000045444F002A
:103DA00045533E00002778000000200000277800DF
:103DB00020E721004FF50700000006001200000078
:103DC000C856410052494100424C450084FA070060
:103DD000ABFF07003CF50700C5FF07000000060029
:103DE00012000000C8434F004E535400414E54008F
:103DF0007BFA0700BBF60700002778006000200070
:103E00000027780000002000D5F4070012F5070015
:103E1000002778000000200097F307006CF10700EE
:103E20000000060022000000C653540052494E0014
:103E3000470000006AFA07000FF10700A9F6070023
:103E4000A8F607000027780060002000002778000F
:103E500000002000C2F40700FFF4070000277800EC
:103E60000000200084F3070059F10700000006005D
:103E700026000000C5564C00495354004BF3070080
:103E800000277800801F78003E0078002000B000F6
:103E900010007800002778004F00780010007800AC
:103EA000FCF00700FBF00700FAF00700F9F007004C
:103EB0001BF40700801F78003E0078003E00780069
:103EC000002778004F00780000277800F0032000DA
:103ED0003E0060000000EA00E6F60700CDF60700AD
:103EE000ECF00700EBF0070000277800000020004E
:103EF000002778002000200056F1070008F4070092
:103F0000E4F00700E3F007003E0070000000B0009E
:103F10003E007800040032004EF1070000277800D0
:103F200000002000040037003E0078003E007800CA
:103F300000277800F0FF2F000000B0003E0078005E
:103F4000D7FF32003E0078003E00780000000600F7
:103F500070000000C34B45005900000063F30700E8
:103F6000002778001000B00014F107000140FE00A7
:103F7000C8F0070011F10700C6F007003E0010006E
:103F80000000B0003E007800F8FF3200C1F00700EA
:103F90003E0040002000B00008F10700801F7800BC
:103FA0003E0078001000B0000027780003F1070001
:103FB0001000B00000277800F00720003E006000ED
:103FC000ADF0070007F10700002778004F007800E8
:103FD0000000060042000000C5494E004B45590054
:103FE00042F3070000277800F4F00700002778006C
:103FF0000027780030002000B4F007001000B00067
:10400000F8F007001000B10000277800F00720004A
:104010003E0060003E0040002000B000E7F00700D6
:104020000000060028000000C84B450059424F0020
:10403000415244002DF307001000B0000027780023
:104040001000B100DDF0070092F00700DBF0070080
:104050003E0010000000B0003E0078000600320074
:1040600000277800D5F007003E0040001000B000A7
:10407000D2F0070002003700002778003E006800F9
:104080000000060030000000C645580050454300BF
:104090005400000000277800F00F20003E00600070
:1040A0000027780000002000002778003000200062
:1040B00086F00700CBF0070076F007001000B00094
:1040C00074F00700002778000002200021F20700AA
:1040D000A2FF07000027780000277800F0012000E9
:1040E00018F107006BF0070000277800F0072000A8
:1040F00008F107003E00600066F007000027780026
:104100009000200009F107003E00700000277800B1
:10411000400020006DF00700A8F00700002778009D
:104120004000200069F00700FAF007003E00600040
:104130000000B0003E007800470032000027780001
:104140000027780090002000F8F007000000B00081
:104150003E007800180032003E007800002778000A
:10416000000220000027780080002000002778004F
:104170004000200055F0070090F00700002778006D
:10418000801F78003E007800002778007000200033
:104190003E0060003E001000002778003000200044
:1041A0004AF00700002778004F0078003E0010001A
:1041B0007CF1070002003700002778001000200083
:1041C000801F78003E00780000277800801F78006C
:1041D0003E00780000277800FEF2070000277800F4
:1041E0003000200039F0070074F007001000B00024
:1041F000002778004000200034F0070079F0070025
:10420000002778003000200030F0070000277800F9
:104210006AF007003E00400072F0070000277800B7
:104220004F007800002778004F0078001000B100A0
:1042300000277800A3F007000000B0003E007800DF
:10424000DFFF32003E0078003E0078000027780053
:10425000000020004F00370000277800002778007A
:10426000F0072000B1F007000AF0070000277800EF
:1042700080002000ADF007003E00700005F0070050
:1042800000277800C0012000A8F007003E00700061
:1042900000277800400020000CF0070047F00700DE
:1042A0008FF007003E0060000000B0003E00780084
:1042B000140032003E007800F6EF07003FF00700E0
:1042C00000277800100020003E0010000027780032
:1042D00030002000FDEF070042F0070000277800C3
:1042E00080002000BBF20700CAF507000027780015
:1042F00080002000B7F207000027780000002000AF
:1043000024003700002778000027780030002000C4
:1043100086F00700DFEF070000277800D0002000BC
:1043200082F007003E007000DAEF070065F007003A
:104330003E0070000000B0003E0078000B0032002C
:104340000027780030002000E0EF07000027780009
:104350001AF007001000B0003E00400021F00700F6
:1043600000277800F0FF2F000A00370000277800B0
:10437000A00020006DF0070079F007000000B000F9
:104380003E007800010032009BF50700002778000E
:10439000000020000000B0003E0078004CFF32001A
:1043A0003E0078003E007800000006009401000006
:1043B000C4515500495400000FD020000027780058
:1043C00000002000002778002BF2070000F0070013
:1043D0002FF20700FEEF070027F207001000780019
:1043E000DDEF07000000B0003E007800150032004D
:1043F000002778004F80DE000000B0003E0078000B
:10440000040032003E00780000277800A00320005E
:104410000B003700002778002000200049F007003B
:104420000000B0003E007800030032000027780052
:1044300020022000020037000027780080022000C0
:104440000200370000277800E003200061F2070037
:104450008BF1070000277800A3F107001000780017
:104460000000B0003E007800030032000027780012
:10447000F00520000200370000277800E00420004B
:1044800004FF070052F507000027780030002000E5
:1044900080EF070000277800C8EF07003E004000CB
:1044A0001000B000CFEF07000027780000002000C8
:1044B00078EF0700CBEF07001000B0008AF107008B
:1044C000100078000000B0003E00780008003200C4
:1044D00000277800300120003EF20700E7FB0700CC
:1044E00000277800100120003AF207000100370091
:1044F000E2FB0700E6F10700100078000000B000C2
:104500003E007800A00032000EE0200076F10700A7
:10451000100078000000B0003E0078000900320072
:10452000C4FE07000000B0003E0078000200320028
:104530008AFE07003E007800002778000000200077
:104540000200370000277800F0FF2F000000B000C5
:104550003E007800EDFF3200C7F107001000780040
:1045600000277800F0FF2F00F0EF07000000B000F8
:104570003E007800200032008CF107000027780010
:10458000801F78003E0078002000B0001000780006
:10459000002778007FB89700100078003DEF0700F3
:1045A0003CEF07003BEF07003AEF070000277800D9
:1045B000000020000027780020002000A5EF070061
:1045C00057F20700A3EF0700002778007FB8970095
:1045D0007FEF0700002778004F0078002000B00030
:1045E0007BEF0700EEF107000027780000002000B5
:1045F000A1F1070076EF070024FA0700052A2A0038
:104600002A2A200025F10700BDF5070019F507004B
:1046100000F507009EF107001000780000277800E1
:104620000027780010002000C0EF07000000B00055
:104630003E0078000A00320014FA0700183A200001
:10464000496E730074727500637469006F6E2000A8
:10465000494E43004F4E4E005545200021747800CE
:10466000002778000027780020002000AFEF070027
:104670000000B0003E0078000A00320003FA070094
:10468000193A2000496E73007472750063746900F2
:104690006F6E2000494D4D0045444900415445008E
:1046A00020217800002778000027780030002000C3
:1046B0009EEF07000000B0003E0078000B003200C3
:1046C000F2F907001B3A200050524F00424C4500BF
:1046D0004D45200050696C00652064006520520043
:1046E00045544F0055522000210D540000277800FA
:1046F00000277800400020008CEF07000000B00089
:104700003E0078000B003200E0F907001D3A20005F
:1047100050524F00424C45004D45200050696C00FE
:104720006520640065732000444F4E004E454500EF
:104730005320210000277800002778004000200047
:1047400080EF07000000B0003E0078000800320053
:10475000CEF907000C3A2000455252004555520050
:10476000206E6F0020696C0079F6070001003700A9
:104770003E007800A0F4070095F4070000277800B9
:10478000F0FF2F000F0037003BF10700100078000A
:104790004CEF07000000B0003E0078000700320038
:1047A00000277800F00420008AF107000027780035
:1047B000B004200087F1070085F407000027780087
:1047C000000020000000B0003E00780002FF320030
:1047D00000277800000020000000B0003E007800B4
:1047E000F5FE3200000006001E020000C541420036
:1047F0004F5254000EE0200097F207000027780087
:10480000000020000027780030F10700F0EE0700DC
:104810000027780026F10700EDEE0700002778005A
:10482000BEF00700EAEE0700C2F00700E8EE07005E
:1048300067F4070095F90700262A2A002A2A200093
:10484000494E54004552520055505400494F4E00B5
:10485000204C6F006769630069656C006C6520001F
:10486000284142004F5254002920210058F40700EB
:1048700061F40700D0FE0700000006000027780062
:104880006003200000277800801F78003E00780039
:1048900010007800002778004F007800002778008B
:1048A0001000200097F0070019F00700C8EE07007D
:1048B00000400600002778006003200000277800F1
:1048C000801F78003E0078001000780000277800F4
:1048D0004F0078000027780010002000B9F0070092
:1048E0000BF0070000277800400820000027780020
:1048F000801F78003E0078001000780000277800C4
:1049000070FF2F003E006000002778004F00780005
:10491000AFEE0700E6F0070010007800E9EE0700B0
:104920000000B0003E0078008C0032006EF00700FE
:10493000100078000000B0003E0078002C0032002B
:1049400069F0070000277800801F78003E0078009B
:10495000100078001000B1000027780000277800D0
:104960004F0078009AEE0700D6EE07000000B00076
:104970003E0078001E003200DCF0070000277800BF
:104980008EEE07001000B00000277800F00720002E
:104990003E0060003FEE07001000B00087EE070009
:1049A0003CEE0700E1EE07000000B0003E0078009A
:1049B000030032003E0078003E0078000C00370013
:1049C00000277800D0002000002778003000200069
:1049D0003EEE07000027780078EE07003E0040001A
:1049E0002000B0007FEE070023EE07007DEE0700F9
:1049F000B6F007001000780078F00700100078008B
:104A0000002778000000B0003E007800510032001E
:104A100020EE07001FEE070010007800B7EE070039
:104A20000000B0003E0078004500320065F007004D
:104A30001000780017EE07002000B000100078008A
:104A4000002778004F80DE00801F78003E0078004D
:104A50003E00100000277800000024003E006000A7
:104A6000002778004F0078003E007000BCEE070081
:104A70000000B0003E0078001700320000277800E8
:104A80001000780091F0070051EE07000027780031
:104A900000002800FFED07002000B0009CEF070099
:104AA000002778004280BF00002778007FF8970039
:104AB000004EB20042E0B7003E007800F5ED07007E
:104AC00003F8070042E0B7003E007800F1ED070070
:104AD0007EF007003EEE07003AF00700811F7800E5
:104AE000821F7800100178009E0078008180E80025
:104AF0001100E0000B003B00210090000000E000EE
:104B00000800320002003B001100100003003700D3
:104B1000000041000001EB00A200980000F0A1009D
:104B2000800878003E0078004F017800CF007800C0
:104B3000200090000027780062EE07000200370096
:104B400000277800F0FF2F000000B0003E00780042
:104B5000AFFF32003E0078003E0078005BF00700B7
:104B600010007800002778002000200063EE070086
:104B70000000B0003E0078003700320026F0070049
:104B800000277800801F78003E0078001000780031
:104B9000002778004F0078002000B0001000780057
:104BA000BCED0700BBED07003E0070000000B00048
:104BB0003E00780026003200002778000000200028
:104BC0000027780014F0070000277800801F780085
:104BD0003E007800FEED0700002778004F007800C7
:104BE0002000B000FAED0700CCEF070010007800BD
:104BF0000000B0003E00780012003200002778006C
:104C0000F00720003E006000002778004F00780089
:104C10000027780000F82F003E0060003E004000B2
:104C2000002778004F0078003E00780092ED0700E2
:104C3000801F78003E007800801F78003E007800DA
:104C4000020037003E0078003E0078000200370086
:104C50003E0078003E007800DDED070000400600D1
:104C6000002778006003200000277800801F78006C
:104C70003E00780010007800002778004F00780090
:104C80000027780020212000CCED070000277800C5
:104C90004008200000277800801F78003E00780040
:104CA0001000780000277800F0DF2F003E00600041
:104CB000002778004F007800C5ED070084EF07005B
:104CC00000277800801F78003E0078002000B000A8
:104CD00010007800002778004F007800100078005E
:104CE0006CED07006BED07003E0070000000B000A7
:104CF0003E007800020032004DF907004600370000
:104D00003E0078003E007800002778001000B100D7
:104D10000000B0003E00780032003200002778002A
:104D2000002778003001200000EE070059ED070051
:104D30000027780010012000FCED07003E00700005
:104D40000000B0003E007800070032000027780025
:104D500030012000F5ED0700E4EF07002008B00067
:104D6000A0ED07001E003700E0EF070000277800E5
:104D700092ED07001000B00000277800F007200037
:104D80003E00600043ED07001000B0008BED07000F
:104D900040ED0700E5ED07000000B0003E007800A0
:104DA000040032003E0078003E0078003E007800AB
:104DB0000B0037003DED0700002778003000200091
:104DC00042ED0700002778007CED07003E00400020
:104DD0002000B00083ED070027ED070081ED0700FC
:104DE0000D003700002778003E006800002778009B
:104DF000603F220088EF070000277800801F7800BE
:104E00003E00780072ED0700002778004F00780020
:104E10002000B0006EED07006DED070000400600B9
:104E20001C030000D15449004D455200315F55002C
:104E300041525400315F49004E4954000027780028
:104E400030992300002778002010200060ED070033
:104E5000002778000000280000277800401020007C
:104E60005BED070000277800700020000027780025
:104E70004021200056ED07000027780000002000A8
:104E80009AEF070052ED0700002778000040280045
:104E900000277800C02020004DED07000027780093
:104EA0000040200000277800E020200048ED0700A7
:104EB000002778008020200000277800C00820000C
:104EC00043ED070000277800000020000DEF0700E9
:104ED0003FED0700000006005C000000C5544500DF
:104EE0004D504F0037EF0700100078000140FE00E2
:104EF000E8EC070033EF0700100078000027780087
:104F000030002000F1EC07003E0010007BED0700B0
:104F10000000B0003E007800F4FF32003E00780050
:104F20003E0078000000060028000000C5464F0043
:104F300052544800D5F70700CA0D45006E74720040
:104F4000657A200064616E0073206C0065206D003E
:104F50006F6E640065206400752046004F52540057
:104F6000480D0D0020202000202043006F707900A4
:104F700072696700687420006A7062002E666F00B4
:104F8000727468000D0D2000204D690063726F007F
:104F900020464F005254480020706F007572200068
:104FA000647350004943330030460D0020566500BD
:104FB000727369006F6E2000312E320032202000A3
:104FC0006475200031362F0031312F00323031002E
:104FD000340D20002068740074703A002F2F6A008E
:104FE00070622E00666F720074682E006672650033
:104FF000652E6600722F0D0020206A0070625F002F
:10500000666F720074684000796168006F6F6700B6
:10501000726F750070732E00636F6D000D0D2000B0
:1050200051756500206C650020464F0052544800C1
:1050300020736F006974200061766500632054005E
:105040004F4921000D0D0D000000060092000000E8
:10505000C6464F005247450054000000D6F40700F2
:105060008CEC07008BEC07003E0070000000B000E5
:105070003E0078001D00320086EC070085EC07003A
:105080000027780000002000002778002000200082
:10509000F0EC07007FEC07007EEC070040EF070014
:1050A0009FEF0700EBEC0700C0EE07000027780039
:1050B000801F78003E007800C5EC070000277800CC
:1050C0004F0078002000B000C1EC070000277800F6
:1050D000F00F200000277800F0FF2F0022EF0700DC
:1050E000B5EF07005CF00700020037003E007800D3
:1050F0003E0078000000060056000000CE54450037
:105100004C4543004841520047454D00454E540030
:10511000E7EE070000277800801F78003E00780047
:105120001000780000277800F0FF2F00002778009B
:105130007FB89700A6EC0700801F78003E0078003B
:105140000027780080BB200067EE0700A0EC070076
:10515000002778004F007800002778004F00780083
:105160009BEC07000000060038000000C944450021
:105170004D4152005241470045000000A0DA200096
:1051800020A0B7000FD020000EE020003CEE07006A
:105190000027780000502000002778000000200041
:1051A000ECED07000027780010002000D6EE070085
:1051B00087EC07000027780080A5200035F0070065
:1051C0001EFF07000CF307000027780000002000F6
:1051D000002778000010200051EF07002DEC070099
:1051E0002CEC070000277800000020000027780042
:1051F0002000200085EC070026EC070025EC0700C6
:1052000047EF0700801F78003E00780000277800F5
:10521000F00F2000C5EC0700002778004F00780051
:1052200000277800F0FF2F00C0EC07003E00600070
:105230000000B0003E007800EAFF320015EC0700E5
:1052400014EC0700D6EE070012EC070000277800E8
:10525000500020001DEC0700B4EC07000DEC070027
:10526000002778005000200018EC0700AFEC070082
:105270003E0060000000B0003E00780005003200F3
:105280003E0078003E00780000277800F0FF2F00F5
:1052900069003700FFEB0700FEEB070000277800EE
:1052A00000002000002778002000200069EC0700A3
:1052B0001BEF0700F7EB07000000B0003E0078008E
:1052C0000A0032003E0078003E0078000027780097
:1052D0000000200000277800200020005DEC07007F
:1052E000002778000000200053003700801F78005E
:1052F0003E007800801F78003E007800E5EB070054
:10530000E4EB0700002778004F00780000277800C2
:105310004F0078004FEC0700DEEB07004F80DE0007
:105320000000B0003E0078000C0032003E00780023
:105330003E00780000277800000020000027780059
:105340002000200043EC0700002778000000200028
:1053500000277800F0FF2F0034003700CDEB070066
:105360000027780070002000D8EB07006FEC0700E2
:10537000C8EB07000027780070002000D3EB07007F
:105380006AEC07003E0060000000B0003E007800BC
:105390000A0032003E0078003E007800C3EB0700B0
:1053A0003E007800C1EB07003E007800002778003F
:1053B000F0FF2F00002778001C003700B5EB070036
:1053C000B4EB0700002778000000200000277800D9
:1053D000200020001FEC0700D1EE0700ADEB070016
:1053E0000000B0003E0078000E0032003E00780061
:1053F0003E0078003E0078003E00780000277800EC
:1054000000002000002778002000200011EC070099
:10541000002778000000200000277800F0FF2F0010
:105420000200370000277800000020000000B000D4
:105430003E007800B7FF32000000B0003E00780068
:1054400081FF320093EB070092EB0700D7ED0700D6
:1054500000277800801F78003E007800DCEB070012
:10546000002778004F0078002000B000D8EB07003C
:1054700088EB070087EB0700A9EE0700801F780084
:105480003E007800002778001004200027EC070079
:10549000002778004F0078000027780050CC2400C7
:1054A00022EC07003E0060000000B0003E007800E3
:1054B000200032000027780000002000002778003C
:1054C00020002000D1EB070072EB070071EB070012
:1054D00093EE0700801F78003E00780000277800D8
:1054E0005004200011EC0700002778004F007800DE
:1054F00000277800E03424000CEC07003E00600038
:105500000000B0003E00780007003200002778005D
:10551000000020000027780020002000BBEB0700DF
:1055200043F70700020037003E0078003E00780095
:10553000020037003E0078003E00780026F20700A7
:105540007CFE07002CF107009BFB07000000060013
:00000001FF
